:100000000C9423010C9497130C9440010C94400120
:100010000C9440010C9440010C9440010C9440015C
:100020000C9440010C9440010C9440010C9440014C
:100030000C9440010C94A2150C943B160C942414BF
:100040000C946E160C946F150C9408160C944001C9
:100050000C94F1130C943C150C94D5150C94981336
:100060000C9440010C94F4090C9440010C94480940
:100070000C9440010C9440020C9440010C944001FB
:100080000C9440010C9440010C9440010C946A14AF
:100090000C941F0A0C9440010C9473090C944001B9
:1000A0000C9440010C9440010C9440010C944001CC
:1000B0000C9440010C94B0140C9440010C94400139
:1000C0000C9440010C9440010C94F6140C944A0AD0
:1000D0000C9440010C949E090C94750A0C944001F8
:1000E0000C94C90907634236B79BD8A71A396856DA
:1000F00018AEBAAB558C1D3CB7CC5763BD6DEDFD4A
:10010000753EF6177231BF000000803F0800000006
:10011000BE922449123EABAAAA2ABECDCCCC4C3EFC
:1001200000000080BEABAAAAAA3E00000000BF00EB
:100130000000803F0000000000084178D3BB4387E7
:10014000D1133D190E3CC3BD4282AD2B3E68EC82FB
:1001500076BED98FE1A93E4C80EFFFBE01C4FF7F80
:100160003F00000000000000010008004000000106
:100170000004000001000800200040008000000191
:1001800000046261644953522063616C6C656400D1
:1001900030313233343536373839414243444546BD
:1001A0000025642025642025642025642025642002
:1001B00025642025642025642025642025642025CD
:1001C000642025642025642025642025642025647E
:1001D0002025642025640D0A0025640D0A004C5F6B
:1001E00053656E736F723D25642C204C5F77686594
:1001F000656C3D256425642C20525F53656E736FDA
:10020000723D25642C20525F776865656C3D2564DE
:1002100025640D0A00496E697469616C697A6174BC
:10022000696F6E20436F6D706C657465200D0A00F8
:100230002E000D0A53797374656D205761726D69D4
:100240006E672055700011241FBECFEFD1E2DEBFD4
:10025000CDBF12E0A0E0B2E0EAE1FEE402C005900A
:100260000D92A639B107D9F715E0A6E9B2E001C0B1
:100270001D92AF35B107E1F70E9487220C940B273E
:100280000C94A116DF93CF93CDB7DEB7AAE7B0E009
:10029000EAE7F0E0808180688C93AAE7B0E0EAE7C3
:1002A000F0E080818F7D8C9386E00E94830181E065
:1002B0000E949701ACE7B0E0ECE7F0E080818F7D31
:1002C0008C93AAE7B0E0EAE7F0E0808188608C9345
:1002D0001092F2047894CF91DF910895DF93CF9339
:1002E000CDB7DEB7AAE7B0E0EAE7F0E08081877F2C
:1002F0008C93AAE7B0E0EAE7F0E080818F778C93F7
:10030000CF91DF910895DF93CF930F92CDB7DEB7F2
:100310008983AAE7B0E0EAE7F0E08081982F987F30
:100320008981892B8C930F90CF91DF910895DF9372
:10033000CF930F92CDB7DEB78983ACE7B0E0ECE79F
:10034000F0E08081282F2F738981882F90E000248E
:10035000969587950794969587950794982F802D65
:10036000822B8C930F90CF91DF910895DF93CF93E1
:100370000F92CDB7DEB78983ACE7B0E0ECE7F0E0F1
:100380008081982F907E89818F71892B8C930F901B
:10039000CF91DF910895DF93CF93CDB7DEB7AAE772
:1003A000B0E0EAE7F0E0808180618C93AAE7B0E0FA
:1003B000EAE7F0E0808180648C93CF91DF9108952B
:1003C000DF93CF93CDB7DEB7EAE7F0E080818074AA
:1003D000CF91DF910895DF93CF930F92CDB7DEB722
:1003E00089831092F2048981883040F0ABE7B0E055
:1003F000EBE7F0E0808188608C9307C0ABE7B0E06A
:10040000EBE7F0E08081877F8C93ACE7B0E0ECE72E
:10041000F0E08081982F987F89818770892B8C9359
:10042000AAE7B0E0EAE7F0E0808180618C93AAE778
:10043000B0E0EAE7F0E0808180648C93EAE7F0E0E6
:100440008081882F90E0807490700097B9F7E8E77A
:10045000F0E0808191810F90CF91DF910895DF933B
:10046000CF930F92CDB7DEB7898389810E94EB01CC
:1004700096958795969587950F90CF91DF910895E2
:100480001F920F920FB60F9211248F93DF93CF9389
:10049000CDB7DEB78FEF8093F204CF91DF918F91CC
:1004A0000F900FBE0F901F901895DF93CF93CDB78D
:1004B000DEB727970FB6F894DEBF0FBECDBF9B8384
:1004C0008A837D836C835F834E83EFE5F0E08081D8
:1004D0008983F894EA81FB818C819D81918380835B
:1004E000EA81FB818E819F8193838283EA81FB81F4
:1004F00017821682EA81FB8115821482EFE5F0E013
:100500008981808327960FB6F894DEBF0FBECDBFDA
:10051000CF91DF910895DF93CF9300D000D0CDB776
:10052000DEB79C838B831A82EFE5F0E080818983BC
:10053000F894EB81FC81848195810097D1F1EB8166
:10054000FC8120813181EB81FC8186819781F901D9
:10055000E80FF91F80818A83EB81FC818681978176
:100560000196EB81FC8197838683EB81FC81268158
:100570003781EB81FC81828193812817390780F0D4
:10058000EB81FC8126813781EB81FC818281938123
:10059000A901481B590BCA01EB81FC819783868313
:1005A000EB81FC81848195810197EB81FC819583AE
:1005B0008483EFE5F0E0898180838A810F900F903A
:1005C0000F900F90CF91DF910895DF93CF9300D0DC
:1005D00000D00F92CDB7DEB79B838A837D836C8377
:1005E000EFE5F0E080818983F894EA81FB81248142
:1005F00035818C819D8182179307B0F5EA81FB815B
:10060000268137818C819D81820F931FEA81FB8136
:1006100097838683EA81FB8126813781EA81FB818A
:10062000828193812817390780F0EA81FB81268136
:100630003781EA81FB8182819381A901481B590B93
:10064000CA01EA81FB8197838683EA81FB81248149
:1006500035818C819D81A901481B590BCA01EA8112
:10066000FB819583848304C0EA81FB811582148217
:10067000EFE5F0E0898180830F900F900F900F904D
:100680000F90CF91DF9108950F931F93DF93CF9336
:1006900000D000D000D0CDB7DEB79C838B837E83A3
:1006A0006D83EFE5F0E080818A83F894EB81FC8133
:1006B00000811181EB81FC81268137818D819E81B2
:1006C000820F931FEB81FC8122813381B9010E944B
:1006D000A726F801E80FF91F80818983EFE5F0E094
:1006E0008A818083898126960FB6F894DEBF0FBE7B
:1006F000CDBFCF91DF911F910F9108950F931F935D
:10070000DF93CF9300D000D00F92CDB7DEB79B839D
:100710008A836C83EFE5F0E080818983F894EA8135
:10072000FB8124813581EA81FB81828193812817B5
:10073000390750F5EA81FB8100811181EA81FB8153
:1007400026813781EA81FB8184819581820F931F05
:10075000EA81FB8122813381B9010E94A726F80139
:10076000E80FF91F8C818083EA81FB818481958168
:100770000196EA81FB8195838483EFE5F0E089812E
:1007800080838FEF8D8305C0EFE5F0E08981808362
:100790001D828D810F900F900F900F900F90CF9131
:1007A000DF911F910F910895DF93CF9300D000D078
:1007B0000F92CDB7DEB79D838C83EFE5F0E08081AB
:1007C0008B83F894EC81FD8122813381EC81FD8162
:1007D00084819581A901481B590BCA019A83898399
:1007E000EFE5F0E08B81808389819A810F900F90F3
:1007F0000F900F900F90CF91DF910895DF93CF93DB
:1008000000D00F92CDB7DEB79B838A83EFE5F0E08F
:1008100080818983F894EA81FB8115821482EFE557
:10082000F0E0898180830F900F900F90CF91DF913E
:100830000895DF93CF93CDB7DEB70E9428040E94BE
:100840004A040E946C040E948E04CF91DF910895A7
:10085000DF93CF93CDB7DEB70E94B0041092D704D8
:100860001092D604E1ECF0E088ED808380E040E86F
:1008700055E260E070E00E9432058FEF8093F30450
:100880001092170510923C0510923B057894CF9179
:10089000DF910895DF93CF93CDB7DEB70E94C904EF
:1008A0001092D9041092D804E9ECF0E088ED80832E
:1008B00081E040E855E260E070E00E9432058FEF91
:1008C0008093F4041092180510923E0510923D0595
:1008D0007894CF91DF910895DF93CF93CDB7DEB7B2
:1008E0000E94E2041092DB041092DA04E1EDF0E0E1
:1008F00088ED808382E040E855E260E070E00E948D
:1009000032058FEF8093F50410921905109240057F
:1009100010923F057894CF91DF910895DF93CF93A4
:10092000CDB7DEB70E94FB041092DD041092DC0408
:10093000E1E3F1E088ED808383E040E855E260E0A8
:1009400070E00E9432058FEF8093F60410921A0532
:1009500010924205109241057894CF91DF9108954D
:10096000DF93CF93CDB7DEB787EF94E026E932E08F
:10097000B90140E850E00E9455028BE195E026E184
:1009800033E0B90140E150E00E945502CF91DF9180
:100990000895DF93CF93CDB7DEB78FEF94E026E2D3
:1009A00033E0B90140E850E00E94550283E295E04F
:1009B00026EA33E0B90140E150E00E945502CF91B0
:1009C000DF910895DF93CF93CDB7DEB787E095E051
:1009D00026EB33E0B90140E850E00E9455028BE27B
:1009E00095E026E334E0B90140E150E00E94550271
:1009F000CF91DF910895DF93CF93CDB7DEB78FE02E
:100A000095E026E434E0B90140E850E00E94550248
:100A100083E395E026EC34E0B90140E150E00E9428
:100A20005502CF91DF910895DF93CF9300D00F92BD
:100A3000CDB7DEB789837B836A838981843060F494
:100A40008981882F90E0880F991FFC01EA52FB4FA3
:100A50008A819B81918380830F900F900F90CF911B
:100A6000DF910895EF92FF920F931F93DF93CF933F
:100A7000CDB7DEB727970FB6F894DEBF0FBECDBF58
:100A80008B834C835D836E837F838C819D81AE815C
:100A9000BF8180589B47A14EBF4F880F991FAA1F47
:100AA000BB1F880F991FAA1FBB1F880F991FAA1F62
:100AB000BB1F7C018D018C819D81AE81BF81880F20
:100AC000991FAA1FBB1F880F991FAA1FBB1F880F42
:100AD000991FAA1FBB1F880F991FAA1FBB1F9C012C
:100AE000AD01C801B7010E94CE26DA01C901019704
:100AF0009A8389838B81833061F4E4E3F1E0898117
:100B00008083E5E3F1E089819A81892F99278083A9
:100B100029C08B81823061F4E4EDF0E0898180832B
:100B2000E5EDF0E089819A81892F992780831AC0A9
:100B30008B81813061F4ECECF0E089818083EDEC15
:100B4000F0E089819A81892F992780830BC0E4EC9A
:100B5000F0E089818083E5ECF0E089819A81892F3A
:100B60009927808327960FB6F894DEBF0FBECDBFBE
:100B7000CF91DF911F910F91FF90EF900895DF9338
:100B8000CF930F92CDB7DEB789838981882F90E00C
:100B9000880F991F880F991F880F991F89509B4FA5
:100BA0000F90CF91DF910895DF93CF930F92CDB740
:100BB000DEB789838981882F90E0880F991F880F7D
:100BC000991F880F991F855E9A4F0F90CF91DF91E3
:100BD0000895DF93CF9300D0CDB7DEB789836A83C2
:100BE0008981833071F4E0E3F1E08081882F90E027
:100BF000807290700097B9F3E6E3F1E08A81808318
:100C00002FC08981823071F4E0EDF0E08081882F7F
:100C100090E0807290700097B9F3E6EDF0E08A8181
:100C200080831EC08981813071F4E8ECF0E080811E
:100C3000882F90E0807290700097B9F3EEECF0E0AE
:100C40008A8180830DC0E0ECF0E08081882F90E005
:100C5000807290700097B9F3E6ECF0E08A818083AF
:100C60008981882F90E0FC01ED50FB4F10820F909E
:100C70000F90CF91DF910895DF93CF930F92CDB76F
:100C8000DEB7898380E069810E94E9050F90CF91EA
:100C9000DF910895DF93CF930F92CDB7DEB78983AD
:100CA00081E069810E94E9050F90CF91DF9108955D
:100CB000DF93CF930F92CDB7DEB7898382E069814E
:100CC0000E94E9050F90CF91DF910895DF93CF93B4
:100CD0000F92CDB7DEB7898383E069810E94E90571
:100CE0000F90CF91DF910895DF93CF9300D00F92B3
:100CF000CDB7DEB780E09E012F5F3F4FB9010E9464
:100D0000F806882331F08981282F30E03B832A833D
:100D100004C08FEF9FEF9B838A838A819B810F9012
:100D20000F900F90CF91DF910895DF93CF9300D074
:100D30000F92CDB7DEB781E09E012F5F3F4FB90123
:100D40000E94F806882331F08981282F30E03B8308
:100D50002A8304C08FEF9FEF9B838A838A819B81C4
:100D60000F900F900F90CF91DF910895DF93CF9365
:100D700000D00F92CDB7DEB782E09E012F5F3F4FCC
:100D8000B9010E94F806882331F08981282F30E0CC
:100D90003B832A8304C08FEF9FEF9B838A838A81E2
:100DA0009B810F900F900F90CF91DF910895DF936B
:100DB000CF9300D00F92CDB7DEB783E09E012F5FB7
:100DC0003F4FB9010E94F806882331F08981282F0E
:100DD00030E03B832A8304C08FEF9FEF9B838A839D
:100DE0008A819B810F900F900F90CF91DF91089592
:100DF000DF93CF9300D000D0CDB7DEB789837B835C
:100E00006A838981882F90E0880F991F880F991F26
:100E10000196880F991FFC01E950FB4F8081918159
:100E2000009731F18981882F90E0880F991F0196F2
:100E3000880F991F880F991FFC01E950FB4F808193
:100E40009181009799F08981882F90E0880F991FF0
:100E5000880F991F880F991F89509B4F0E948B0202
:100E6000EA81FB8180838FEF8C8303C01C8201C0E9
:100E70001C828C810F900F900F900F90CF91DF917B
:100E80000895DF93CF930F92CDB7DEB78983898121
:100E9000882F90E0880F991F880F991F880F991F3E
:100EA00089509B4F0E94FE030F90CF91DF910895D0
:100EB000DF93CF9300D0CDB7DEB789838981882FA8
:100EC00090E0880F991F0196880F991F880F991F2E
:100ED000FC01E950FB4F808191811A82009711F447
:100EE00081E08A838A810F900F90CF91DF910895DE
:100EF000DF93CF9300D0CDB7DEB789836A83898132
:100F0000882F90E0880F991F880F991F880F991FCD
:100F1000855E9A4F6A810E947E030F900F90CF9159
:100F2000DF910895DF93CF930F92CDB7DEB789831A
:100F300080E069810E9478070F90CF91DF9108953A
:100F4000DF93CF930F92CDB7DEB7898381E06981BC
:100F50000E9478070F90CF91DF910895DF93CF9390
:100F60000F92CDB7DEB7898382E069810E9478074E
:100F70000F90CF91DF910895DF93CF930F92CDB76C
:100F8000DEB7898383E069810E9478070F90CF9153
:100F9000DF910895DF93CF930F92CDB7DEB78983AA
:100FA0008981882F90E0FC01E95EFA4F8FEF808302
:100FB0008981882F90E0880F991F880F991F880FCB
:100FC000991F855E9A4F0E948B02982F8981692F05
:100FD0000E94E9050F90CF91DF910895DF93CF93A1
:100FE000CDB7DEB729970FB6F894DEBF0FBECDBFE1
:100FF00089837B836A835D834C838981882F90E01A
:10100000880F991F0196880F991F880F991FFC015F
:10101000E55EFA4F208131818C819D81280F391F37
:101020008981882F90E0880F991F880F991F01965A
:10103000880F991FFC01E55EFA4F80819181281786
:10104000390708F045C08C819D81009709F440C0A4
:10105000EA81FB81208128878A819B8101969B837D
:101060008A831F821E821DC08981882F90E0880F8D
:10107000991F880F991F880F991F9C01255E3A4F71
:10108000EA81FB8140818A819B8101969B838A83CF
:10109000C901642F0E947E038E819F8101969F83E8
:1010A0008E838C819D8101972E813F81281739077E
:1010B000D8F28981882F90E0FC01E95EFA4F8FEF2A
:1010C0008083898168850E94E9053FEF398701C0E7
:1010D0001986898529960FB6F894DEBF0FBECDBF5D
:1010E000CF91DF9108950F931F93DF93CF930F92CA
:1010F000CDB7DEB789838981882F90E0FC01E95E56
:10110000FA4F8081882309F44EC08981882F90E0AE
:10111000880F991F0196880F991F880F991FFC014E
:10112000E55EFA4F80819181009769F18981833072
:1011300049F406E311E083E395E00E948B02F80195
:10114000808339C08981823049F406ED10E08BE25A
:1011500095E00E948B02F80180832DC08981813047
:1011600049F40EEC10E083E295E00E948B02F80156
:10117000808321C006EC10E08BE195E00E948B0299
:10118000F801808318C08981882F90E0FC01E95E16
:10119000FA4F10828981882F90E0FC01ED50FB4FBF
:1011A0008FEF808308C08981882F90E0FC01ED508B
:1011B000FB4F8FEF80830F90CF91DF911F910F91A5
:1011C0000895DF93CF9300D0CDB7DEB78A838A81AD
:1011D000833029F4E6E3F1E08081898314C08A81B9
:1011E000823029F4E6EDF0E0808189830CC08A81A9
:1011F000813029F4EEECF0E08081898304C0E6ECD4
:10120000F0E0808189838A81882F90E0880F991F80
:10121000FC01EA52FB4F80819181009771F08A8135
:10122000882F90E0880F991FFC01EA52FB4F019034
:10123000F081E02D8981099526C08A81882F90E070
:10124000880F991F880F991F880F991F89509B4FEE
:1012500069810E947E038823B1F48A81282F30E0BF
:10126000C901880F991FFC01E55CFA4F80819181CB
:10127000AC014F5F5F4FC901880F991FFC01E55C0E
:10128000FA4F518340830F900F90CF91DF910895D3
:101290001F920F920FB60F9211242F933F934F93EB
:1012A0005F936F937F938F939F93AF93BF93EF93CE
:1012B000FF93DF93CF93CDB7DEB780E00E94730832
:1012C000CF91DF91FF91EF91BF91AF919F918F915E
:1012D0007F916F915F914F913F912F910F900FBE32
:1012E0000F901F9018951F920F920FB60F92112416
:1012F0002F933F934F935F936F937F938F939F931E
:10130000AF93BF93EF93FF93DF93CF93CDB7DEB748
:1013100081E00E947308CF91DF91FF91EF91BF911F
:10132000AF919F918F917F916F915F914F913F917D
:101330002F910F900FBE0F901F9018951F920F9234
:101340000FB60F9211242F933F934F935F936F9398
:101350007F938F939F93AF93BF93EF93FF93DF930D
:10136000CF93CDB7DEB782E00E947308CF91DF91B3
:10137000FF91EF91BF91AF919F918F917F916F916D
:101380005F914F913F912F910F900FBE0F901F9043
:1013900018951F920F920FB60F9211242F933F931F
:1013A0004F935F936F937F938F939F93AF93BF936D
:1013B000EF93FF93DF93CF93CDB7DEB783E00E9427
:1013C0007308CF91DF91FF91EF91BF91AF919F9102
:1013D0008F917F916F915F914F913F912F910F90DE
:1013E0000FBE0F901F9018951F920F920FB60F927D
:1013F00011242F933F934F935F936F937F938F931A
:101400009F93AF93BF93EF93FF93DF93CF93CDB7AA
:10141000DEB780E00E94E108CF91DF91FF91EF916C
:10142000BF91AF919F918F917F916F915F914F91FC
:101430003F912F910F900FBE0F901F9018951F9204
:101440000F920FB60F9211242F933F934F935F93F8
:101450006F937F938F939F93AF93BF93EF93FF937C
:10146000DF93CF93CDB7DEB781E00E94E108CF9143
:10147000DF91FF91EF91BF91AF919F918F917F91FC
:101480006F915F914F913F912F910F900FBE0F90F1
:101490001F9018951F920F920FB60F9211242F9341
:1014A0003F934F935F936F937F938F939F93AF93EC
:1014B000BF93EF93FF93DF93CF93CDB7DEB782E077
:1014C0000E94E108CF91DF91FF91EF91BF91AF9121
:1014D0009F918F917F916F915F914F913F912F914C
:1014E0000F900FBE0F901F9018951F920F920FB67E
:1014F0000F9211242F933F934F935F936F937F939A
:101500008F939F93AF93BF93EF93FF93DF93CF930B
:10151000CDB7DEB783E00E94E108CF91DF91FF9164
:10152000EF91BF91AF919F918F917F916F915F915B
:101530004F913F912F910F900FBE0F901F901895D4
:10154000DF93CF9300D000D000D0CDB7DEB79C831F
:101550008B838B819C81039625E030E0B9010E944A
:10156000A726CB01CC01A0E0B0E0880F991FAA1FED
:10157000BB1F880F991FAA1FBB1F880F991FAA1F87
:10158000BB1F880F991FAA1FBB1F9A8389831E82C6
:101590001D8206C02D813E812F5F3F4F3E832D83EC
:1015A00089819A812D813E812817390798F32696E3
:1015B0000FB6F894DEBF0FBECDBFCF91DF91089577
:1015C000DF93CF930F92CDB7DEB7198206C0898122
:1015D0000E94FB0C89818F5F898389818730B8F3F2
:1015E0000E94010B0E94170B0E942C0B0E94420BC1
:1015F0000E94590B0E94700B78940F90CF91DF914D
:101600000895DF93CF93CDB7DEB785E00E94870BB7
:10161000E6E4F0E01082AEE6B0E0EEE6F0E08081D5
:1016200081608C930E94E80DCF91DF910895DF9344
:10163000CF93CDB7DEB783E00E949B0BE4E8F0E0E8
:1016400011821082AFE6B0E0EFE6F0E080818160C9
:101650008C93CF91DF910895DF93CF93CDB7DEB711
:1016600084E00E94AF0BE2EBF0E01082A0E7B0E074
:10167000E0E7F0E0808181608C930E94280ECF919A
:10168000DF910895DF93CF93CDB7DEB783E00E945B
:10169000C30BE4E9F0E011821082A1E7B0E0E1E7DA
:1016A000F0E0808181608C930E94480ECF91DF91A1
:1016B0000895DF93CF93CDB7DEB783E00E94D70BB9
:1016C000E4EAF0E011821082A2E7B0E0E2E7F0E0A5
:1016D000808181608C930E94680ECF91DF91089584
:1016E000DF93CF93CDB7DEB783E00E94EB0BE4E24C
:1016F000F1E011821082A3E7B0E0E3E7F0E080813F
:1017000081608C930E94880ECF91DF910895DF93C2
:10171000CF930F92CDB7DEB78983A5E4B0E0E5E4BF
:10172000F0E08081982F987F8981892B8C930F908E
:10173000CF91DF910895DF93CF930F92CDB7DEB7AE
:101740008983A1E8B0E0E1E8F0E08081982F987FFC
:101750008981892B8C930F90CF91DF910895DF932E
:10176000CF930F92CDB7DEB78983A1EBB0E0E1EB69
:10177000F0E08081982F987F8981892B8C930F903E
:10178000CF91DF910895DF93CF930F92CDB7DEB75E
:101790008983A1E9B0E0E1E9F0E08081982F987FAA
:1017A0008981892B8C930F90CF91DF910895DF93DE
:1017B000CF930F92CDB7DEB78983A1EAB0E0E1EA1B
:1017C000F0E08081982F987F8981892B8C930F90EE
:1017D000CF91DF910895DF93CF930F92CDB7DEB70E
:1017E0008983A1E2B1E0E1E2F1E08081982F987F66
:1017F0008981892B8C930F90CF91DF910895DF938E
:10180000CF9300D000D0CDB7DEB7E5E4F0E0808123
:10181000882F90E087709070880F991F8A599E4F8B
:101820009C838B838B819C81FC01859194919A830D
:101830008983FC83EB8389819A810F900F900F90AD
:101840000F90CF91DF910895DF93CF9300D000D018
:10185000CDB7DEB7E1E8F0E08081882F90E08770B7
:101860009070880F991F8A599E4F9C838B838B8120
:101870009C81FC01859194919A838983FC83EB83FD
:1018800089819A810F900F900F900F90CF91DF91E7
:101890000895DF93CF9300D000D0CDB7DEB7E1EB52
:1018A000F0E08081882F90E087709070880F991FFA
:1018B0008E589E4F9C838B838B819C81FC018591EC
:1018C00094919A838983FC83EB8389819A810F9019
:1018D0000F900F900F90CF91DF910895DF93CF93EA
:1018E00000D000D0CDB7DEB7E1E9F0E08081882FED
:1018F00090E087709070880F991F8E589E4F9C8340
:101900008B838B819C81FC01859194919A8389833F
:10191000FC83EB8389819A810F900F900F900F9039
:10192000CF91DF910895DF93CF9300D000D0CDB752
:10193000DEB7E1EAF0E08081882F90E08770907058
:10194000880F991F8E589E4F9C838B838B819C811F
:10195000FC01859194919A838983FC83EB8389812F
:101960009A810F900F900F900F90CF91DF91089573
:10197000DF93CF9300D000D0CDB7DEB7E1E2F1E046
:101980008081882F90E087709070880F991F8E5803
:101990009E4F9C838B838B819C81FC0185919491CC
:1019A0009A838983FC83EB8389819A810F900F90BE
:1019B0000F900F90CF91DF910895DF93CF9300D0D8
:1019C0000F92CDB7DEB789837B836A8389818730A5
:1019D00060F48981882F90E0880F991FFC01E25202
:1019E000FB4F8A819B81918380830F900F900F9092
:1019F000CF91DF910895DF93CF930F92CDB7DEB7EC
:101A000089838981873050F48981882F90E0880FFD
:101A1000991FFC01E252FB4F118210820F90CF916F
:101A2000DF910895EF92FF920F931F93DF93CF936F
:101A3000CDB7DEB72F970FB6F894DEBF0FBECDBF80
:101A40009B878A87E6E4F0E08081898710924B05C6
:101A500010924C0510924D0510924E050E94FF0BFE
:101A60009C0140E050E080E094E2A4EFB0E0BC01D3
:101A7000CD010E94F026DA01C9018D839E83AF83D8
:101A8000B8878D819E81AF81B885893B2DE892070B
:101A900026E0A20720E0B20720F58A859B85A7E211
:101AA00081319A07F0F48A859B85CC01A0E0B0E0F3
:101AB0002D813E814F815885BC01CD010E94882631
:101AC000DC01CB0128EE33E040E050E0BC01CD0169
:101AD0000E94CE26DA01C90189839A83AB83BC8335
:101AE0003EC08A859B857C0100E010E08D819E814F
:101AF000AF81B88528EE33E040E050E0BC01CD0175
:101B00000E94CE26DA01C9019C01AD01C801B701CE
:101B10000E948826DC01CB0189839A83AB83BC8336
:101B20001EC080914B0590914C05A0914D05B09140
:101B30004E05A3E5B0E0E3E5F0E08081817F8C9382
:101B4000A3E5B0E0E3E5F0E0808181608C938895C7
:101B5000A3E5B0E0E3E5F0E080818E7F8C93809197
:101B60004B0590914C05A0914D05B0914E05222753
:101B7000382F492F5A2FE6E4F0E08081882F90E03B
:101B8000A0E0B0E079018A01E82AF92A0A2B1B2B90
:101B90008985282F30E040E050E089819A81AB812F
:101BA000BC81820F931FA41FB51FE816F9060A0710
:101BB0001B0708F4B6CF2F960FB6F894DEBF0FBE02
:101BC000CDBFCF91DF911F910F91FF90EF900895BE
:101BD000DF93CF93CDB7DEB710924705109248053B
:101BE0001092490510924A05CF91DF910895DF9335
:101BF000CF93CDB7DEB78091470590914805A0916E
:101C00004905B0914A05BC01CD01CF91DF910895FE
:101C1000DF93CF93CDB7DEB71092530510925405E2
:101C20001092550510925605CF91DF910895DF93DC
:101C3000CF93CDB7DEB78091530590915405A09115
:101C40005505B0915605BC01CD01CF91DF910895A6
:101C5000DF93CF93CDB7DEB710924F0510925005AA
:101C60001092510510925205CF91DF910895DF93A4
:101C7000CF93CDB7DEB780914F0590915005A091DD
:101C80005105B0915205BC01CD01CF91DF9108956E
:101C9000DF93CF93CDB7DEB710925B0510925C0552
:101CA00010925D0510925E05CF91DF910895DF934C
:101CB000CF93CDB7DEB780915B0590915C05A09185
:101CC0005D05B0915E05BC01CD01CF91DF91089516
:101CD000DF93CF93CDB7DEB7109243051092440542
:101CE0001092450510924605CF91DF910895DF933C
:101CF000CF93CDB7DEB78091430590914405A09175
:101D00004505B0914605BC01CD01CF91DF91089505
:101D1000DF93CF93CDB7DEB71092570510925805D9
:101D20001092590510925A05CF91DF910895DF93D3
:101D3000CF93CDB7DEB78091570590915805A0910C
:101D40005905B0915A05BC01CD01CF91DF9108959D
:101D5000DF93CF930F92CDB7DEB789838981893026
:101D600079F4A0E8B0E0E0E8F0E0808182608C9354
:101D7000A0E8B0E0E0E8F0E080818E7F8C9320C0A6
:101D800089818A3079F4A0E8B0E0E0E8F0E0808171
:101D900082608C93A0E8B0E0E0E8F0E080818160B0
:101DA0008C930EC0A0E8B0E0E0E8F0E080818D7F89
:101DB0008C93A0E8B0E0E0E8F0E0808181608C9353
:101DC000EAE8F0E0118210820F90CF91DF91089540
:101DD000DF93CF930F92CDB7DEB7898389818930A6
:101DE00079F4A0EBB0E0E0EBF0E0808182608C93CE
:101DF000A0EBB0E0E0EBF0E080818E7F8C9320C020
:101E000089818A3079F4A0EBB0E0E0EBF0E08081EA
:101E100082608C93A0EBB0E0E0EBF0E08081816029
:101E20008C930EC0A0EBB0E0E0EBF0E080818D7F02
:101E30008C93A0EBB0E0E0EBF0E0808181608C93CC
:101E4000E4EBF0E010820F90CF91DF910895DF93E3
:101E5000CF930F92CDB7DEB789838981893079F42A
:101E6000A0E9B0E0E0E9F0E0808182608C93A0E935
:101E7000B0E0E0E9F0E080818E7F8C9320C0898122
:101E80008A3079F4A0E9B0E0E0E9F0E08081826096
:101E90008C93A0E9B0E0E0E9F0E0808181608C9370
:101EA0000EC0A0E9B0E0E0E9F0E080818D7F8C9386
:101EB000A0E9B0E0E0E9F0E0808181608C93E8E99E
:101EC000F0E0118210820F90CF91DF910895DF939F
:101ED000CF930F92CDB7DEB789838981893079F4AA
:101EE000A1E9B0E0E1E9F0E0808182608C93A1E9B2
:101EF000B0E0E1E9F0E080818E7F8C9320C08981A1
:101F00008A3079F4A1E9B0E0E1E9F0E08081826013
:101F10008C93A1E9B0E0E1E9F0E0808181608C93ED
:101F20000EC0A1E9B0E0E1E9F0E080818D7F8C9303
:101F3000A1E9B0E0E1E9F0E0808181608C93EAE919
:101F4000F0E0118210820F90CF91DF910895DF931E
:101F5000CF930F92CDB7DEB789838981893079F429
:101F6000A2E9B0E0E2E9F0E0808182608C93A2E92E
:101F7000B0E0E2E9F0E080818E7F8C9320C089811F
:101F80008A3079F4A2E9B0E0E2E9F0E08081826091
:101F90008C93A2E9B0E0E2E9F0E0808181608C936B
:101FA0000EC0A2E9B0E0E2E9F0E080818D7F8C9381
:101FB000A2E9B0E0E2E9F0E0808181608C93ECE995
:101FC000F0E0118210820F90CF91DF910895DF939E
:101FD000CF930F92CDB7DEB789838981893079F4A9
:101FE000A0EAB0E0E0EAF0E0808182608C93A0EAB1
:101FF000B0E0E0EAF0E080818E7F8C9320C08981A0
:102000008A3079F4A0EAB0E0E0EAF0E08081826012
:102010008C93A0EAB0E0E0EAF0E0808181608C93EC
:102020000EC0A0EAB0E0E0EAF0E080818D7F8C9302
:10203000A0EAB0E0E0EAF0E0808181608C93E8EA19
:10204000F0E0118210820F90CF91DF910895DF931D
:10205000CF930F92CDB7DEB789838981893079F428
:10206000A1EAB0E0E1EAF0E0808182608C93A1EA2D
:10207000B0E0E1EAF0E080818E7F8C9320C089811E
:102080008A3079F4A1EAB0E0E1EAF0E08081826090
:102090008C93A1EAB0E0E1EAF0E0808181608C936A
:1020A0000EC0A1EAB0E0E1EAF0E080818D7F8C9380
:1020B000A1EAB0E0E1EAF0E0808181608C93EAEA95
:1020C000F0E0118210820F90CF91DF910895DF939D
:1020D000CF930F92CDB7DEB789838981893079F4A8
:1020E000A0EAB0E0E0EAF0E0808182608C93A0EAB0
:1020F000B0E0E0EAF0E080818E7F8C9320C089819F
:102100008A3079F4A0EAB0E0E0EAF0E08081826011
:102110008C93A0EAB0E0E0EAF0E0808181608C93EB
:102120000EC0A0EAB0E0E0EAF0E080818D7F8C9301
:10213000A0EAB0E0E0EAF0E0808181608C93ECEA14
:10214000F0E0118210820F90CF91DF910895DF931C
:10215000CF9300D0CDB7DEB79A838983A0E8B0E0F3
:10216000E0E8F0E080818E7F8C93A0E8B0E0E0E8CA
:10217000F0E0808182608C93A1E8B0E0E1E8F0E0DB
:10218000808188608C93A1E8B0E0E1E8F0E0808194
:1021900080618C93E6E8F0E089819A819183808365
:1021A000E8E8F0E011821082EAE8F0E011821082A3
:1021B000ECE8F0E0118210820F900F90CF91DF9148
:1021C0000895DF93CF9300D0CDB7DEB79A8389838C
:1021D000A0E9B0E0E0E9F0E080818E7F8C93A0E997
:1021E000B0E0E0E9F0E0808182608C93A1E9B0E0AA
:1021F000E1E9F0E0808188608C93A1E9B0E0E1E959
:10220000F0E0808180618C93E6E9F0E089819A8139
:1022100091838083E8E9F0E011821082EAE9F0E03E
:1022200011821082ECE9F0E0118210820F900F9081
:10223000CF91DF910895DF93CF9300D0CDB7DEB774
:102240009A838983A0EAB0E0E0EAF0E080818E7FA3
:102250008C93A0EAB0E0E0EAF0E0808182608C93A9
:10226000A1EAB0E0E1EAF0E0808188608C93A1EA25
:10227000B0E0E1EAF0E0808180618C93E6EAF0E092
:1022800089819A8191838083E8EAF0E0118210824B
:10229000EAEAF0E011821082ECEAF0E011821082AA
:1022A0000F900F90CF91DF910895DF93CF93CDB72B
:1022B000DEB7A0E8B0E0E0E8F0E0808180628C93D7
:1022C000A0E8B0E0E0E8F0E080818F7E8C93CF91D1
:1022D000DF910895DF93CF93CDB7DEB7A0EBB0E0E9
:1022E000E0EBF0E0808180628C93A0EBB0E0E0EB6B
:1022F000F0E080818F7E8C93CF91DF910895DF9302
:10230000CF93CDB7DEB7A0E9B0E0E0E9F0E080819F
:1023100080688C93A0E9B0E0E0E9F0E080818F7BF9
:102320008C93CF91DF910895DF93CF93CDB7DEB734
:10233000A0E9B0E0E0E9F0E0808180628C93A0E960
:10234000B0E0E0E9F0E080818F7E8C93CF91DF9167
:102350000895DF93CF93CDB7DEB7A0E9B0E0E0E911
:10236000F0E0808188608C93A0E9B0E0E0E9F0E0E3
:1023700080818B7F8C93CF91DF910895DF93CF93F2
:10238000CDB7DEB7A0EAB0E0E0EAF0E08081806897
:102390008C93A0EAB0E0E0EAF0E080818F7B8C9340
:1023A000CF91DF910895DF93CF93CDB7DEB7A0EA49
:1023B000B0E0E0EAF0E0808180628C93A0EAB0E0D7
:1023C000E0EAF0E080818F7E8C93CF91DF910895D9
:1023D000DF93CF93CDB7DEB7A0EAB0E0E0EAF0E05C
:1023E000808188608C93A0EAB0E0E0EAF0E0808130
:1023F0008B7F8C93CF91DF910895DF93CF93CDB7EF
:10240000DEB7A0E8B0E0E0E8F0E080818F7D8C935B
:10241000A0E8B0E0E0E8F0E080818F7E8C93CF917F
:10242000DF910895DF93CF93CDB7DEB7A0EBB0E097
:10243000E0EBF0E080818F7D8C93A0EBB0E0E0EBEF
:10244000F0E080818F7E8C93CF91DF910895DF93B0
:10245000CF93CDB7DEB7A0E9B0E0E0E9F0E080814E
:102460008F778C93A0E9B0E0E0E9F0E080818F7B8A
:102470008C93CF91DF910895DF93CF93CDB7DEB7E3
:10248000A0E9B0E0E0E9F0E080818F7D8C93A0E9E5
:10249000B0E0E0E9F0E080818F7E8C93CF91DF9116
:1024A0000895DF93CF93CDB7DEB7A0E9B0E0E0E9C0
:1024B000F0E08081877F8C93A0E9B0E0E0E9F0E074
:1024C00080818B7F8C93CF91DF910895DF93CF93A1
:1024D000CDB7DEB7A0EAB0E0E0EAF0E080818F7728
:1024E0008C93A0EAB0E0E0EAF0E080818F7B8C93EF
:1024F000CF91DF910895DF93CF93CDB7DEB7A0EAF8
:10250000B0E0E0EAF0E080818F7D8C93A0EAB0E05B
:10251000E0EAF0E080818F7E8C93CF91DF91089587
:10252000DF93CF93CDB7DEB7A0EAB0E0E0EAF0E00A
:102530008081877F8C93A0EAB0E0E0EAF0E08081C0
:102540008B7F8C93CF91DF910895DF93CF93CDB79D
:10255000DEB7A0E8B0E0E0E8F0E080818D7F8C930A
:10256000A0E8B0E0E0E8F0E080818E7F8C930E94EC
:10257000FD11CF91DF910895DF93CF93CDB7DEB7F3
:10258000A0EBB0E0E0EBF0E080818D7F8C93A0EBDE
:10259000B0E0E0EBF0E080818E7F8C930E9412121D
:1025A000CF91DF910895DF93CF93CDB7DEB7A0E948
:1025B000B0E0E0E9F0E080818D7F8C93A0E9B0E0AD
:1025C000E0E9F0E080818E7F8C930E9427120E94C8
:1025D0003C120E945112CF91DF910895DF93CF9367
:1025E000CDB7DEB7A0EAB0E0E0EAF0E080818D7F11
:1025F0008C93A0EAB0E0E0EAF0E080818E7F8C93DB
:102600000E9466120E947B120E949012CF91DF916D
:102610000895DF93CF9300D0CDB7DEB79A83898337
:10262000EAE8F0E089819A81918380830F900F908E
:10263000CF91DF910895DF93CF9300D0CDB7DEB770
:102640009A838983E4EBF0E0898180830F900F9077
:10265000CF91DF910895DF93CF9300D0CDB7DEB750
:102660009A838983E8E9F0E089819A819183808364
:102670000F900F90CF91DF910895DF93CF9300D00B
:10268000CDB7DEB79A838983EAE9F0E089819A8140
:10269000918380830F900F90CF91DF910895DF9306
:1026A000CF9300D0CDB7DEB79A838983ECE9F0E011
:1026B00089819A81918380830F900F90CF91DF91D0
:1026C0000895DF93CF9300D0CDB7DEB79A83898387
:1026D000E8EAF0E089819A81918380830F900F90DE
:1026E000CF91DF910895DF93CF9300D0CDB7DEB7C0
:1026F0009A838983EAEAF0E089819A8191838083D1
:102700000F900F90CF91DF910895DF93CF9300D07A
:10271000CDB7DEB79A838983ECEAF0E089819A81AC
:10272000918380830F900F90CF91DF91089518953A
:102730001F920F920FB60F9211242F933F934F9336
:102740005F936F937F938F939F93AF93BF93EF9319
:10275000FF93DF93CF93CDB7DEB78091470590917C
:102760004805A0914905B0914A050196A11DB11DEA
:102770008093470590934805A0934905B0934A0577
:1027800080914B0590914C05A0914D05B0914E055F
:102790000196A11DB11D80934B0590934C05A0930C
:1027A0004D05B0934E058091DE049091DF040097B3
:1027B00029F0E091DE04F091DF040995CF91DF91DB
:1027C000FF91EF91BF91AF919F918F917F916F9109
:1027D0005F914F913F912F910F900FBE0F901F90DF
:1027E00018951F920F920FB60F9211242F933F93BB
:1027F0004F935F936F937F938F939F93AF93BF9309
:10280000EF93FF93DF93CF93CDB7DEB78091E004D2
:102810009091E104009729F0E091E004F091E10447
:102820000995CF91DF91FF91EF91BF91AF919F916A
:102830008F917F916F915F914F913F912F910F9069
:102840000FBE0F901F9018951F920F920FB60F9208
:1028500011242F933F934F935F936F937F938F93A5
:102860009F93AF93BF93EF93FF93DF93CF93CDB736
:10287000DEB780914F0590915005A0915105B09120
:1028800052050196A11DB11D80934F0590935005EF
:10289000A0935105B09352058091E8049091E9040A
:1028A000009729F0E091E804F091E9040995CF91AF
:1028B000DF91FF91EF91BF91AF919F918F917F91A8
:1028C0006F915F914F913F912F910F900FBE0F909D
:1028D0001F9018951F920F920FB60F9211242F93ED
:1028E0003F934F935F936F937F938F939F93AF9398
:1028F000BF93EF93FF93DF93CF93CDB7DEB7809174
:102900005B0590915C05A0915D05B0915E05019617
:10291000A11DB11D80935B0590935C05A0935D059F
:10292000B0935E058091F0049091F104009729F036
:10293000E091F004F091F1040995CF91DF91FF91BE
:10294000EF91BF91AF919F918F917F916F915F9127
:102950004F913F912F910F900FBE0F901F901895A0
:102960001F920F920FB60F9211242F933F934F9304
:102970005F936F937F938F939F93AF93BF93EF93E7
:10298000FF93DF93CF93CDB7DEB78091430590914E
:102990004405A0914505B09146050196A11DB11DC4
:1029A0008093430590934405A0934505B093460555
:1029B0008091F2049091F304009729F0E091F204E1
:1029C000F091F3040995CF91DF91FF91EF91BF91C1
:1029D000AF919F918F917F916F915F914F913F91B7
:1029E0002F910F900FBE0F901F9018951F920F926E
:1029F0000FB60F9211242F933F934F935F936F93D2
:102A00007F938F939F93AF93BF93EF93FF93DF9346
:102A1000CF93CDB7DEB78091570590915805A0911F
:102A20005905B0915A050196A11DB11D8093570516
:102A300090935805A0935905B0935A058091F404DA
:102A40009091F504009729F0E091F404F091F504D9
:102A50000995CF91DF91FF91EF91BF91AF919F9138
:102A60008F917F916F915F914F913F912F910F9037
:102A70000FBE0F901F9018951F920F920FB60F92D6
:102A800011242F933F934F935F936F937F938F9373
:102A90009F93AF93BF93EF93FF93DF93CF93CDB704
:102AA000DEB78091F6049091F704009729F0E09149
:102AB000F604F091F7040995CF91DF91FF91EF9122
:102AC000BF91AF919F918F917F916F915F914F9146
:102AD0003F912F910F900FBE0F901F9018951F924E
:102AE0000F920FB60F9211242F933F934F935F9342
:102AF0006F937F938F939F93AF93BF93EF93FF93C6
:102B0000DF93CF93CDB7DEB78091E2049091E304D9
:102B1000009729F0E091E204F091E3040995CF9148
:102B2000DF91FF91EF91BF91AF919F918F917F9135
:102B30006F915F914F913F912F910F900FBE0F902A
:102B40001F9018951F920F920FB60F9211242F937A
:102B50003F934F935F936F937F938F939F93AF9325
:102B6000BF93EF93FF93DF93CF93CDB7DEB7809101
:102B7000FC049091FD04009729F0E091FC04F09191
:102B8000FD040995CF91DF91FF91EF91BF91AF9136
:102B90009F918F917F916F915F914F913F912F9175
:102BA0000F900FBE0F901F9018951F920F920FB6A7
:102BB0000F9211242F933F934F935F936F937F93C3
:102BC0008F939F93AF93BF93EF93FF93DF93CF9335
:102BD000CDB7DEB78091F8049091F904009729F001
:102BE000E091F804F091F9040995CF91DF91FF91FC
:102BF000EF91BF91AF919F918F917F916F915F9175
:102C00004F913F912F910F900FBE0F901F901895ED
:102C10001F920F920FB60F9211242F933F934F9351
:102C20005F936F937F938F939F93AF93BF93EF9334
:102C3000FF93DF93CF93CDB7DEB78091E4049091FB
:102C4000E504009729F0E091E404F091E50409958A
:102C5000CF91DF91FF91EF91BF91AF919F918F91B4
:102C60007F916F915F914F913F912F910F900FBE88
:102C70000F901F9018951F920F920FB60F9211246C
:102C80002F933F934F935F936F937F938F939F9374
:102C9000AF93BF93EF93FF93DF93CF93CDB7DEB79F
:102CA0008091FE049091FF04009729F0E091FE04CA
:102CB000F091FF040995CF91DF91FF91EF91BF91C2
:102CC000AF919F918F917F916F915F914F913F91C4
:102CD0002F910F900FBE0F901F9018951F920F927B
:102CE0000FB60F9211242F933F934F935F936F93DF
:102CF0007F938F939F93AF93BF93EF93FF93DF9354
:102D0000CF93CDB7DEB78091E6049091E7040097AA
:102D100029F0E091E604F091E7040995CF91DF9165
:102D2000FF91EF91BF91AF919F918F917F916F91A3
:102D30005F914F913F912F910F900FBE0F901F9079
:102D400018951F920F920FB60F9211242F933F9355
:102D50004F935F936F937F938F939F93AF93BF93A3
:102D6000EF93FF93DF93CF93CDB7DEB782E891E087
:102D700000D00F92EDB7FEB7319621E02083928309
:102D800081830E9459190F900F900F90CF91DF917E
:102D9000FF91EF91BF91AF919F918F917F916F9133
:102DA0005F914F913F912F910F900FBE0F901F9009
:102DB0001895DF93CF9300D0CDB7DEB79A83898380
:102DC00089819A819093ED048093EC040F900F9089
:102DD000CF91DF910895DF93CF930F92CDB7DEB7F8
:102DE000898389818A3031F4E091EC04F091ED041B
:102DF0008DE00995E091EC04F091ED04898109954D
:102E00000F90CF91DF910895DF93CF9300D0CDB78E
:102E1000DEB79A83898389819A81009789F00BC0F4
:102E2000E981FA81208189819A8101969A83898337
:102E3000822F0E94EB16E981FA818081882381F735
:102E40000F900F90CF91DF910895DF93CF93CDB77F
:102E5000DEB72A970FB6F894DEBF0FBECDBF9A83B8
:102E600089837C836B835E834D8318861F8289816F
:102E70009A81009709F449C02F81388519868B8182
:102E80009C812817390710F481E089878F81988504
:102E9000019698878F8381E099858927882391F40B
:102EA000E981FA8180818A878A85882311F091E0FF
:102EB0009A878A8529813A812F5F3F4F3A832983F8
:102EC0008823D1F618861F8219C0E981FA81808192
:102ED000882361F0E981FA81208189819A810196B4
:102EE0009A838983822F0E94EB1603C080E20E949E
:102EF000EB168F819885019698878F832F8138856F
:102F00008D819E812817390700F32A960FB6F89411
:102F1000DEBF0FBECDBFCF91DF910895DF93CF937A
:102F200000D000D000D0CDB7DEB79D838C838C81DC
:102F30009D810097B1F003C08E810E94EB168C81B9
:102F40009D819B838A838C819D8101969D838C8347
:102F5000EA81FB818491898389818E838E81882394
:102F600059F726960FB6F894DEBF0FBECDBFCF91AE
:102F7000DF910895DF93CF93CDB7DEB78AE00E944B
:102F8000EB16CF91DF910895DF93CF9300D000D05F
:102F9000CDB7DEB78C838C81882F90E08F709070D6
:102FA00080579E4F9B838A83EA81FB81849189832A
:102FB00089810E94EB160F900F900F900F90CF9188
:102FC000DF910895DF93CF930F92CDB7DEB789835A
:102FD000898182958F700E94C41789810E94C417CD
:102FE0000F90CF91DF910895DF93CF9300D0CDB7AD
:102FF000DEB79A83898389819A81892F99270E94D4
:10300000E21789810E94E2170F900F90CF91DF9114
:103010000895DF93CF9300D000D0CDB7DEB769839A
:103020007A838B839C8389819A81AB81BC81CD011A
:10303000AA27BB270E94F41789819A810E94F4175E
:103040000F900F900F900F90CF91DF910895EF9216
:10305000FF920F931F93DF93CF93CDB7DEB7E8971F
:103060000FB6F894DEBF0FBECDBF8EA76FA748ABDB
:1030700029ABEAAAFBAA0CAB1DAB88A98823B1F047
:103080008AA99BA9ACA9BDA9BB2384F48AA99BA941
:10309000ACA9BDA9B095A095909581959F4FAF4FD4
:1030A000BF4F88879987AA87BB8708C08AA99BA931
:1030B000ACA9BDA988879987AA87BB8788A98EAB49
:1030C0008EA9882311F081E08EAB9EA98FA5891B64
:1030D00081508F83CE010E9680969D878C878C853C
:1030E0009D8501979D878C87EC85FD8510828C8559
:1030F0009D8501979D878C878EA5282F30E040E025
:1031000050E088859985AA85BB85BC01CD010E94C8
:10311000CE26DC01CB018F70907080579E4F9E832E
:103120008D83ED81FE8184918C838C81EC85FD857E
:1031300080838EA5282F30E040E050E08885998577
:10314000AA85BB85BC01CD010E94CE26DA01C9014A
:1031500088879987AA87BB8747C088859985AA856C
:10316000BB850097A105B105B1F18C859D850197BF
:103170009D878C878EA5282F30E040E050E0888521
:103180009985AA85BB85BC01CD010E94CE26DC01B4
:10319000CB018F70907080579E4F9B838A83EA810A
:1031A000FB81849189838981EC85FD8580838EA54F
:1031B000282F30E040E050E088859985AA85BB85BE
:1031C000BC01CD010E94CE26DA01C901888799870A
:1031D000AA87BB8709C08C859D8501979D878C87B1
:1031E000EC85FD8589A980838F818FAB8FA988238A
:1031F00011F081E08FAB8FA99F8191509F8388232D
:1032000009F0ABCF88A9882361F18AA99BA9ACA951
:10321000BDA9BB2354F48C859D8501979D878C8720
:10322000EC85FD858DE280831CC08AA99BA9ACA991
:10323000BDA9181619061A061B0654F48C859D851F
:1032400001979D878C87EC85FD858BE2808309C083
:103250008C859D8501979D878C87EC85FD8580E217
:1032600080838FA58F830BC0EC85FD8520818C85A5
:103270009D8501969D878C87822F0E94EB168F81FA
:1032800088AF88AD882311F081E088AF88AD9F8139
:1032900091509F83882341F7E8960FB6F894DEBFDC
:1032A0000FBECDBFCF91DF911F910F91FF90EF9097
:1032B0000895DF93CF93CDB7DEB763970FB6F89439
:1032C000DEBF0FBECDBFCE014B969F878E8711C04C
:1032D0008D85882359F480E090E063960FB6F894CA
:1032E000DEBF0FBECDBFCF91DF9108958D850E94C7
:1032F000EB16888D882381F0898D9A8D9E838D832E
:10330000898D9A8D01969A8F898FED81FE818491A6
:103310008C838C818B8B09C0E98DFA8D20812B8B5E
:10332000898D9A8D01969A8F898F3B893D878D85EE
:10333000853271F6888D882381F0898D9A8D9B83E3
:103340008A83898D9A8D01969A8F898FEA81FB8174
:103350008491898389818A8B09C0E98DFA8D808166
:103360008A8B898D9A8D01969A8F898F9A899D87EC
:103370008D85282F30E0398B288B88899989843670
:103380009105C1F02889398928373105E1F088890C
:1033900099898336910551F42E853F85C90102969E
:1033A0009F878E87F901808191818D878D850E940D
:1033B000EB169FCF8AE090E098878F8380E197E2B9
:1033C0009A87898708C080E190E098878F8380E0A2
:1033D00090E19A8789872E853F85C90102969F874C
:1033E0008E87F901808191819C878B878D858436BA
:1033F00029F58B859C859923ACF48B859C859095CC
:1034000081959F4F9C878B878DE20E94EB160AC0A7
:1034100089859A852AE030E0B9010E94A726CB0170
:103420009A87898789859A858230910538F0298520
:103430003A858B859C858217930750F38B859C85F5
:1034400029853A85B9010E94A726CB010E94C4179D
:103450008B859C8529853A85B9010E94A7269C8782
:103460008B8789859A852F813885B9010E94A72687
:10347000CB019A87898789859A850097F9F639CF94
:10348000DF93CF93CDB7DEB7E0E3F0E01082E1E366
:10349000F0E01082E7E0F1E01082E8E0F1E0108275
:1034A000E1E2F0E08FEF8083E4E2F0E080E480830B
:1034B000E7E2F0E08FEF8083EAE2F0E08BEF8083D9
:1034C000EDE2F0E08EEF8083A4E3B0E0E4E3F0E02F
:1034D000808180628C93A3E3B0E0E3E3F0E080813D
:1034E0008F7D8C93E1E0F1E08EEF8083E4E0F1E00A
:1034F0008EEF8083CF91DF910895DF93CF9300D03B
:1035000000D0CDB7DEB769837A838B839C830BC0F1
:1035100089819A81AB81BC810197A109B109898315
:103520009A83AB83BC8389819A81AB81BC810097EC
:10353000A105B10569F70F900F900F900F90CF91F3
:10354000DF910895DF93CF93CDB7DEB7A5E2B0E06A
:10355000E5E2F0E0808180648C93CF91DF91089563
:10356000DF93CF93CDB7DEB7A5E2B0E0E5E2F0E0C0
:1035700080818F7B8C93CF91DF910895DF93CF93E0
:10358000CDB7DEB7E6E4F0E010820E94E80DCF91FF
:10359000DF910895DF93CF93CDB7DEB7E4E8F0E095
:1035A000118210820E94080ECF91DF910895DF935F
:1035B000CF93CDB7DEB7E2EBF0E010820E94280E89
:1035C000CF91DF910895DF93CF93CDB7DEB7E4E9D4
:1035D000F0E0118210820E94480ECF91DF91089591
:1035E000DF93CF93CDB7DEB7E4EAF0E0118210822B
:1035F0000E94680ECF91DF910895DF93CF93CDB7EE
:10360000DEB7E4E2F1E0118210820E94880ECF91D1
:10361000DF910895DF93CF9300D0CDB7DEB7E2E31B
:10362000F0E08081882F90E0807290701A82198279
:10363000009721F481E090E09A83898389819A81BF
:103640000F900F90CF91DF910895DF93CF9300D02B
:1036500000D000D0CDB7DEB769837A838B839C839B
:1036600089819A81AB81BC81BB23C4F089819A8115
:10367000AB81BC8125E030E040E050E0BC01CD01F1
:103680000E94F026DA01C901880F991FFC01E05061
:10369000FE4F208131813E832D832CC089819A8108
:1036A000AB81BC81B095A095909581959F4FAF4F10
:1036B000BF4F25E030E040E050E0BC01CD010E946A
:1036C000F026DA01C9019C01AD0188E490E0A0E098
:1036D000B0E0821B930BA40BB50B880F991FFC0164
:1036E000E050FE4F8081918122273327281B390B20
:1036F0003E832D838D819E8126960FB6F894DEBF82
:103700000FBECDBFCF91DF910895DF93CF9300D04F
:1037100000D000D0CDB7DEB769837A838B839C83DA
:1037200089819A81AB81BC818A559040A040B0408C
:1037300089839A83AB83BC8389819A81AB81BC8165
:10374000BB23C4F089819A81AB81BC8125E030E044
:1037500040E050E0BC01CD010E94F026DA01C90131
:10376000880F991FFC01E050FE4F208131813E837C
:103770002D832CC089819A81AB81BC81B095A095A5
:10378000909581959F4FAF4FBF4F25E030E040E0CF
:1037900050E0BC01CD010E94F026DA01C9019C0174
:1037A000AD0188E490E0A0E0B0E0821B930BA40B95
:1037B000B50B880F991FFC01E050FE4F808191816D
:1037C00022273327281B390B3E832D838D819E8131
:1037D00026960FB6F894DEBF0FBECDBFCF91DF9116
:1037E00008950F931F93DF93CF9300D000D000D0A4
:1037F000CDB7DEB769837A838B839C8389819A8175
:10380000AB81BC818A359105A105B10521F1898182
:103810009A81AB81BC81863A2FEF92072FEFA207E6
:103820002FEFB207C1F089819A81AB81BC818E30C4
:1038300041E0940740E0A40740E0B40761F08981CB
:103840009A81AB81BC81823F5EEF95075FEFA50750
:103850005FEFB50719F41E821D8224C089819A8109
:10386000AB81BC81BC01CD010E94851B8C0189818B
:103870009A81AB81BC81BC01CD010E94251B9C01BA
:10388000C801B9010E94BB26CB019C01220F331F46
:10389000C901880F991F880F991FA901480F591F47
:1038A0005E834D838D819E8126960FB6F894DEBF90
:1038B0000FBECDBFCF91DF911F910F910895DF9380
:1038C000CF9300D0CDB7DEB79A83898389819A815F
:1038D000AA2797FDA095BA2FBC01CD010E94CA234B
:1038E000DC01CB01BC01CD012BE531EB4FE75FEBF8
:1038F0000E94B924DC01CB01BC01CD012DEC3CE0E0
:103900004DEA54E40E945624DC01CB01BC01CD01F8
:103910000E949723DC01CB010F900F90CF91DF9194
:103920000895DF93CF9300D0CDB7DEB79A83898314
:1039300089819A81AA2797FDA095BA2FBC01CD0154
:103940000E94CA23DC01CB01BC01CD012AE037ED86
:1039500043E65FEB0E94B924DC01CB01BC01CD0141
:1039600020E030E14EEE54E40E945624DC01CB010D
:10397000BC01CD010E949723DC01CB010F900F9079
:10398000CF91DF910895DF93CF9300D0CDB7DEB70D
:103990009A83898389819A81AA2797FDA095BA2F56
:1039A000BC01CD010E94CA23DC01CB01BC01CD01C9
:1039B0002EEE3CE74FE45FEB0E94B924DC01CB0123
:1039C000BC01CD0122E538ED48E354E40E945624C1
:1039D000DC01CB01BC01CD010E949723DC01CB01AE
:1039E0000F900F90CF91DF910895DF93CF9300D088
:1039F000CDB7DEB79A83898389819A81AA2797FDFB
:103A0000A095BA2FBC01CD010E94CA23DC01CB01D5
:103A1000BC01CD0128EA37E54AE65FEB0E94B924F4
:103A2000DC01CB01BC01CD0124EA30EF4EEF53E4C1
:103A30000E945624DC01CB01BC01CD010E949723DA
:103A4000DC01CB010F900F90CF91DF910895DF93B0
:103A5000CF9300D0CDB7DEB79A83898389819A81CD
:103A6000AA2797FDA095BA2FBC01CD010E94CA23B9
:103A7000DC01CB01BC01CD012FE93DEC4AE45FEB59
:103A80000E94B924DC01CB01BC01CD0121E73DE05E
:103A900048E354E40E945624DC01CB01BC01CD0173
:103AA0000E949723DC01CB010F900F90CF91DF9103
:103AB0000895DF93CF9300D0CDB7DEB79A83898383
:103AC00089819A81AA2797FDA095BA2FBC01CD01C3
:103AD0000E94CA23DC01CB01BC01CD0127EA38EEEC
:103AE00042E051E40E945624DC01CB01BC01CD012F
:103AF00027EA38EE42E051E40E943223DC01CB0198
:103B0000BC01CD010E949723DC01CB010F900F90E7
:103B1000CF91DF910895DF93CF9300D0CDB7DEB77B
:103B20009A83898389819A81AA2797FDA095BA2FC4
:103B3000BC01CD010E94CA23DC01CB01BC01CD0137
:103B400027EA38EE42E051E40E945624DC01CB0122
:103B5000BC01CD0127EA38EE42E051E40E94322355
:103B6000DC01CB01BC01CD010E949723DC01CB011C
:103B70000F900F90CF91DF910895DF93CF9300D0F6
:103B8000CDB7DEB79A83898329813A81C901880F2D
:103B9000991F820F931F9C01220F331F220F331F87
:103BA000820F931F845B90400F900F90CF91DF9115
:103BB0000895DF93CF9300D0CDB7DEB79A83898382
:103BC00089819A81AA2797FDA095BA2FBC01CD01C2
:103BD0000E94CA23DC01CB01BC01CD012DE33AE0F8
:103BE00048E452E40E945624DC01CB01BC01CD0123
:103BF0002BE734E14CE452E40E943223DC01CB0198
:103C0000BC01CD010E949723DC01CB010F900F90E6
:103C1000CF91DF910895DF93CF93CDB7DEB7A1E2C7
:103C2000B0E0E1E2F0E0808188608C93A2E2B0E055
:103C3000E2E2F0E08081877F8C9382E090E00E9456
:103C4000A00AA2E2B0E0E2E2F0E0808188608C931A
:103C500085E090E00E94A00AA2E2B0E0E2E2F0E09B
:103C60008081877F8C93A1E2B0E0E1E2F0E0908177
:103C700088E089278C93E0E2F0E08081882F90E053
:103C8000887090700097B9F30E94BE1AE0E2F0E0ED
:103C90008081882F90E0887090700097B9F70E941B
:103CA000F70DDC01CB012FEF30E040E050E0BC012C
:103CB000CD010E9488269B01AC01E6E4F0E0808102
:103CC000882F90E0A0E0B0E0820F931FA41FB51FE3
:103CD000BC01CD010E94CA23DC01CB01BC01CD0196
:103CE0002EEE39E644E050E40E945624DC01CB017C
:103CF000BC01CD010E949723DC01CB01CF91DF9164
:103D00000895DF93CF9300D0CDB7DEB79A83898330
:103D100089819A81AA2797FDA095BA2FBC01CD0170
:103D20000E94CA23DC01CB01BC01CD0120E030E0C0
:103D300040E85EE30E945624DC01CB01BC01CD01CA
:103D400020E030E040E251E40E943323DC01CB016B
:103D5000BC01CD010E949723DC01CB010F900F9095
:103D6000CF91DF910895DF93CF9300D0CDB7DEB729
:103D70009A83898389819A81845F9140AA2797FDDC
:103D8000A095BA2FBC01CD010E94CA23DC01CB0152
:103D9000BC01CD012FE832EC45E75DE30E945624DB
:103DA000DC01CB01BC01CD010E949723DC01CB01DA
:103DB0000F900F90CF91DF910895DF93CF9300D0B4
:103DC000CDB7DEB79A83898324EF31E089819A8168
:103DD000A901481B590BCA010F900F90CF91DF9199
:103DE0000895DF93CF9300D000D0CDB7DEB79A838C
:103DF000898389819A81885C90409C838B838B81A5
:103E00009C8199232CF48B819C8103969C838B83CA
:103E10008B819C8195958795959587950F900F90AF
:103E20000F900F90CF91DF910895DF93CF9300D043
:103E3000CDB7DEB79A83898389819A81845F914067
:103E4000AA2797FDA095BA2FBC01CD010E94CA23D5
:103E5000DC01CB01BC01CD0120E030E040E05EE3BD
:103E60000E945624DC01CB01BC01CD010E949723A6
:103E7000DC01CB010F900F90CF91DF910895DF937C
:103E8000CF9300D0CDB7DEB79A83898389819A8199
:103E9000AA2797FDA095BA2FBC01CD010E94CA2385
:103EA000DC01CB01BC01CD0120E030E040E85DE366
:103EB0000E945624DC01CB01BC01CD010E94972356
:103EC000DC01CB010F900F90CF91DF910895DF932C
:103ED000CF9300D0CDB7DEB79A83898389819A8149
:103EE000845F9140AA2797FDA095BA2FBC01CD0110
:103EF0000E94CA23DC01CB01BC01CD012DEC3CECBE
:103F00004CE45DE30E945624DC01CB01BC01CD01F1
:103F10000E949723DC01CB010F900F90CF91DF918E
:103F20000895DF93CF9300D0CDB7DEB79A8389830E
:103F300089819A81AA2797FDA095BA2FBC01CD014E
:103F40000E94CA23DC01CB01BC01CD012DEC3CEC6D
:103F50004CEC5CE30E945624DC01CB01BC01CD019A
:103F60000E949723DC01CB010F900F90CF91DF913E
:103F70000895DF93CF9300D0CDB7DEB79A838983BE
:103F800089819A81AA2797FDA095BA2FBC01CD01FE
:103F90000E94CA23DC01CB01BC01CD0129E335E439
:103FA00047E45EE30E945624DC01CB01BC01CD0155
:103FB00025E83BEE47E252E40E943223DC01CB01CC
:103FC000BC01CD010E949723DC01CB010F900F9023
:103FD000CF91DF910895DF93CF9300D000D0CDB77C
:103FE000DEB79A8389837C836B8382E040E056E965
:103FF00060E070E00E94320589810E9458068B8142
:104000000E9458060F900F900F900F90CF91DF9164
:104010000895DF93CF9300D0CDB7DEB79A8389831D
:1040200082E040E056E960E070E00E94320589815C
:104030000E9458060F900F90CF91DF9108950F9333
:104040001F93DF93CF93CDB7DEB7A0970FB6F89449
:10405000DEBF0FBECDBF85E00E9483010E94D71A4C
:1040600080E00E942F02882F90E098A38F8F81E03C
:104070000E942F02882F90E09E8F8D8F82E00E94F9
:104080002F02882F90E09C8F8B8F83E00E942F025D
:10409000882F90E09A8F898F84E00E942F02882FCA
:1040A00090E0988F8F8B85E00E942F02882F90E000
:1040B0009E8B8D8B86E00E942F02882F90E09C8B38
:1040C0008B8B87E00E942F02882F90E09A8B898B40
:1040D00088E00E942F02882F90E0988B8F8789E0DC
:1040E0000E942F02882F90E09E878D878AE00E9491
:1040F0002F02882F90E09C878B878BE00E942F02F5
:10410000882F90E09A8789878CE00E942F02882F61
:1041100090E098878F838DE00E942F02882F90E097
:104120009E838D838EE00E942F02882F90E09C83D7
:104130008B838FE00E942F02882F90E09A838983DF
:1041400001EA11E00E94370EDC01CB012FEF30E0D5
:1041500040E050E0BC01CD010E9488269B01AC01EB
:10416000E2EBF0E08081882F90E0A0E0B0E0280F43
:10417000391F4A1F5B1F8DB79EB787970FB6F894FC
:104180009EBF0FBE8DBFEDB7FEB7319681E0808335
:10419000128301838F8D98A1948383838D8D9E8D4F
:1041A000968385838B8D9C8D90878783898D9A8D4F
:1041B000928781878F89988D948783878D899E893F
:1041C000968785878B899C89908B878789899A892F
:1041D000928B818B8F859889948B838B8D859E851F
:1041E000968B858B8B859C85908F878B89859A850F
:1041F000928F818F8F819885948F838F8D819E81FF
:10420000968F858F8B819C8190A3878F89819A81DE
:1042100092A381A323A334A345A356A30E945919B3
:104220008DB79EB787960FB6F8949EBF0FBE8DBF11
:1042300015CFDF93CF9300D0CDB7DEB782E00E94D9
:10424000830189E00E942F02882F90E09A8389835E
:1042500029ED31E000D000D00F92EDB7FEB73196D6
:1042600081E080833283218389819A81948383834F
:104270000E9459190F900F900F900F900F90E1CF5F
:10428000DF93CF93CDB7DEB70E946E21CF91DF9140
:104290000895DF93CF93CDB7DEB782E00E942F025F
:1042A000282F30E08091F0049091F104820F931F49
:1042B00090939502809394028EE00E942F02282F03
:1042C00030E08091EE049091EF04820F931F909361
:1042D000930280939202CF91DF910895DF93CF9361
:1042E000CDB7DEB72A970FB6F894DEBF0FBECDBFAD
:1042F00084EF91E0A0E0B0E08F839887A987BA8728
:1043000084EF91E0A0E0B0E08B839C83AD83BE831B
:1043100088E090E09A8389830E944921209192024B
:1043200030919302809194029091950282179307A5
:1043300088F420919202309193028091940290919E
:104340009502A901481B590BCA019093F10480936F
:10435000F00410C020919402309195028091920255
:1043600090919302A901481B590BCA019093EF0445
:104370008093EE040E944921209192023091930291
:1043800080919402909195028217930700F52091F5
:104390009202309193028091940290919502281B91
:1043A000390B89819A818217930788F486E292E01B
:1043B000A0E0B0E08F839887A987BA8786E292E071
:1043C000A0E0B0E08B839C83AD83BE833BC0209193
:1043D00094023091950280919202909193028217FB
:1043E000930700F5209194023091950280919202FA
:1043F00090919302281B390B89819A818217930728
:1044000088F482E593E0A0E0B0E08F839887A987E5
:10441000BA8782E593E0A0E0B0E08B839C83AD8314
:10442000BE8310C088E592E0A0E0B0E08F8398875B
:10443000A987BA8780E293E0A0E0B0E08B839C83F9
:10444000AD83BE832EED31E04091920250919302F4
:1044500060919402709195028DB79EB70F970FB639
:10446000F8949EBF0FBE8DBFEDB7FEB7319681E0C9
:10447000808332832183548343838F819885A985E8
:10448000BA8585839683A783B087728761878B817E
:104490009C81AD81BE8183879487A587B6870E9462
:1044A00059194DB75EB7415F5F4F0FB6F8945EBFC5
:1044B0000FBE4DBFAEE2B0E0EEE2F0E0808180647E
:1044C0008C938F819885A985BA85BC01CD010E9406
:1044D0007D1AAEE2B0E0EEE2F0E080818F7B8C935B
:1044E000A8E2B0E0E8E2F0E0808180688C938B8104
:1044F0009C81AD81BE81BC01CD010E947D1AA8E2E4
:10450000B0E0E8E2F0E080818F778C9333CFDF93E7
:10451000CF9300D000D0CDB7DEB71C821B821A82A9
:1045200019820E94190480E040E056E960E070E0E2
:104530000E94320581E040E052EC61E070E00E94B0
:10454000320582E040E056E960E070E00E9432050A
:1045500083E040E056E960E070E00E9432058AE4C2
:1045600096E00E94D9160E94401A0E94B01A22E3D7
:1045700032E000D00F92EDB7FEB7319681E0808334
:10458000328321830E9459190F900F900F900E943F
:10459000010B0E94170B0E942C0B0E94420B0E94E1
:1045A000590B0E94420185E00E94830181E00E9434
:1045B00097011C821B8222C08B810E942F02882FB0
:1045C00090E09A83898368E873E180E090E00E943C
:1045D0007D1A20E332E000D00F92EDB7FEB731969E
:1045E00081E08083328321830E9459190F900F90BC
:1045F0000F908B819C8101969C838B838B819C8106
:1046000080319105CCF20E94A21A85E192E000D09F
:104610000F92EDB7FEB7319621E02083928381831C
:104620000E9459190F900F900F900E940A1B00973B
:10463000E1F30E9419210E940A1B0097E1F30E94F6
:10464000BE1A0E94CA1A0E94D71A0E94E31A0E9438
:10465000F01A0E94402164E670E080E090E00E9441
:104660007D1AF7CF5058BB27AA270ED0E5C0D6D069
:1046700030F0DBD020F031F49F3F11F41EF4CBC0BA
:104680000EF4E095E7FBC1C0E92FE7D080F3BA173D
:10469000620773078407950718F071F49EF5FFC051
:1046A0000EF4E0950B2EBA2FA02D0B01B90190014D
:1046B0000C01CA01A0011124FF27591B99F0593F91
:1046C00050F4503E68F11A16F040A22F232F342FD9
:1046D0004427585FF3CF469537952795A795F04027
:1046E0005395C9F77EF41F16BA0B620B730B840B3C
:1046F000BAF09150A1F0FF0FBB1F661F771F881FF4
:10470000C2F70EC0BA0F621F731F841F48F487954B
:1047100077956795B795F7959E3F08F0B3CF93953A
:10472000880F08F09927EE0F97958795089504D084
:104730006894B111B5C0089598D088F09F5790F053
:10474000B92F9927B751A0F0D1F0660F771F881FB6
:10475000991F1AF0BA95C9F712C0B13081F09FD0F5
:10476000B1E008959CC0672F782F8827B85F39F093
:10477000B93FCCF3869577956795B395D9F73EF415
:1047800090958095709561957F4F8F4F9F4F0895BD
:10479000E89409C097FB3EF49095809570956195DB
:1047A0007F4F8F4F9F4F9923A9F0F92F96E9BB2791
:1047B0009395F695879577956795B795F111F8CF0D
:1047C000FAF4BB0F11F460FF1BC06F5F7F4F8F4F78
:1047D0009F4F16C0882311F096E911C0772321F06E
:1047E0009EE8872F762F05C0662371F096E8862F06
:1047F00070E060E02AF09A95660F771F881FDAF75D
:10480000880F9695879597F9089597F99F6780E89F
:1048100070E060E008959FEF80EC089500240A9412
:104820001616170618060906089500240A9412168B
:104830001306140605060895092E0394000C11F4BE
:10484000882352F0BB0F40F4BF2B11F460FF04C06B
:104850006F5F7F4F8F4F9F4F089557FD9058440FC4
:10486000551F59F05F3F71F04795880F97FB991FCF
:1048700061F09F3F79F0879508951216130614068C
:10488000551FF2CF4695F1DF08C016161706180619
:10489000991FF1CF86957105610508940895E894F4
:1048A000BB2766277727CB0197F908950BD0C4CF94
:1048B000B5DF28F0BADF18F0952309F0A6CFABCF0B
:1048C0001124EECFCADFA0F3959FD1F3950F50E0EE
:1048D000551F629FF001729FBB27F00DB11D639FB2
:1048E000AA27F00DB11DAA1F649F6627B00DA11D58
:1048F000661F829F2227B00DA11D621F739FB00DFE
:10490000A11D621F839FA00D611D221F749F33276D
:10491000A00D611D231F849F600D211D822F762F06
:104920006A2F11249F5750408AF0E1F088234AF003
:10493000EE0FFF1FBB1F661F771F881F915050404F
:10494000A9F79E3F510570F060CFAACF5F3FECF30F
:10495000983EDCF3869577956795B795F795E7953B
:104960009F5FC1F7FE2B880F911D9695879597F94C
:104970000895FA01EE0FFF1F30962105310599F1D8
:104980006115710561F48038BFE39B0749F16894B4
:104990009038810561F08038BFEF9B0741F0992383
:1049A00042F5FF3FE1053105210511F1E894089436
:1049B000E795D901AA2329F4AB2FBE2FF85FD0F3D6
:1049C00010C0FF5F70F4A695E0F7F73950F019F0CA
:1049D000FF3A38F49F779F930CD00F9007FC9058C4
:1049E00008953EF018CF60E070E080E89FE30895FE
:1049F0004FE79F775F934F933F932F939ED02F91D5
:104A00003F914F915F9152DF05C019F40EF0FDCE3A
:104A100046CF01CF2ADFC8F39638C0F707F80F92C8
:104A2000E8942BE33AEA48EB5FE74EDF0F920F92F0
:104A30000F924DB75EB70F92C0D0E4EEF0E016D003
:104A40004F915F91EF91FF91E595EE1FFF1F49F0A8
:104A5000FE57E0684427EE0F441FFA95E1F74195B1
:104A6000550B32D00F9007FE26C00895DF93CF93E9
:104A70001F930F93FF92EF92DF927B018C0168945A
:104A800005C0DA2EEF011EDFFE01E894A591259105
:104A9000359145915591AEF3EF01F6DDFE01970199
:104AA000A801DA9479F7DF90EF90FF900F911F91B2
:104AB000CF91DF9108959B01AC0160E070E080E848
:104AC0009FE3AEC0A2CE14C1D0DEE8F39923D9F3A0
:104AD000940F511DBBF39150504094F059F088232E
:104AE00032F0660F771F881F91505040C1F79E3FEC
:104AF000510544F7880F911D9695879597F908956C
:104B00005F3FACF0983E9CF0BB2786957795679504
:104B1000B79508F4B1609395C1F7BB0F58F711F43E
:104B200060FFE8CF6F5F7F4F8F4F9F4FE3CFB8CECF
:104B30000EF0DEC070CE689468CE97DEC8F399237D
:104B4000D1F3C6F3DF93CF931F930F93FF92C92F37
:104B5000DD2788232AF02197660F771F881FDAF751
:104B600020E030E040E85FEB9FE3883920F0803EB2
:104B700030F021968F7777DDECE0F1E003C073DD54
:104B8000E9E3F1E073DF8B01BE01EC01FB2E6F570F
:104B900071097595771F880B990BFCDD28E132E7C9
:104BA00041E35FE38FDEAF2D9801AE01FF900F91DF
:104BB0001F91CF91DF9168DD3FCEFA01DC01AA0F92
:104BC000BB1F9B01AC01BF5728F422273327442782
:104BD00050781FC0B75188F4AB2F00244695379505
:104BE0002795011CA395D2F3002069F0220F331FF3
:104BF000441FB395DAF30DD035CD61307105A0E8CF
:104C00008A07B94630F49B01AC01662777278827CD
:104C10009078309621F02083318342835383089526
:104C20000CD00ACE02DE40F0F9DD30F021F45F3F17
:104C300019F0EBCD511134CEEECD0FDE98F3992360
:104C4000C9F35523B1F3951B550BBB27AA27621750
:104C50007307840738F09F5F5F4F220F331F441F95
:104C6000AA1FA9F333D00E2E3AF0E0E830D09150CD
:104C70005040E695001CCAF729D0FE2F27D0660FBA
:104C8000771F881FBB1F261737074807AB07B0E8F9
:104C900009F0BB0B802DBF01FF2793585F4F2AF00F
:104CA0009E3F510568F0B1CDFBCD5F3FECF3983EE0
:104CB000DCF3869577956795B795F7959F5FC9F76C
:104CC000880F911D9695879597F90895E1E0660FF5
:104CD000771F881FBB1F621773078407BA0720F06E
:104CE000621B730B840BBA0BEE1F88F7E0950895D7
:104CF0009F3F49F0915028F4869577956795B79531
:104D00009F5F80389F4F880F9695879597F90895F4
:104D1000629FD001739FF001829FE00DF11D649F9F
:104D2000E00DF11D929FF00D839FF00D749FF00D2B
:104D3000659FF00D9927729FB00DE11DF91F639FCC
:104D4000B00DE11DF91FBD01CF0111240895AA1B6B
:104D5000BB1B51E107C0AA1FBB1FA617B70710F066
:104D6000A61BB70B881F991F5A95A9F78095909598
:104D7000BC01CD01089597FB092E07260AD077FDC7
:104D800004D0E5DF06D000201AF4709561957F4FBE
:104D90000895F6F7909581959F4F0895A1E21A2EF8
:104DA000AA1BBB1BFD010DC0AA1FBB1FEE1FFF1FCF
:104DB000A217B307E407F50720F0A21BB30BE40B1F
:104DC000F50B661F771F881F991F1A9469F7609566
:104DD0007095809590959B01AC01BD01CF01089520
:104DE00097FB092E05260ED057FD04D0D7DF0AD039
:104DF000001C38F450954095309521953F4F4F4F0A
:104E00005F4F0895F6F790958095709561957F4F67
:0A4E10008F4F9F4F0895F894FFCFD5
:104E1A0064006400620061005E005B00570052009B
:104E2A004D0047004000390032002A0022001A00D3
:104E3A00110009000000F7FFEFFFE6FFDEFFD6FFD3
:104E4A00CEFFC7FFC0FFB9FFB3FFAEFFA9FFA5FFA3
:104E5A00A2FF9FFF9EFF9CFF9CFF9CFF9EFF9FFF60
:104E6A00A2FFA5FFA9FFAEFFB3FFB9FFC0FFC7FFAF
:104E7A00CEFFD6FFDEFFE6FFEFFFF7FF00000900D7
:104E8A0011001A0022002A003200390040004700AF
:104E9A004D00520057005B005E0061006200640032
:064EAA006400800080009E
:00000001FF
